:1000000000308A00A42800000A108A100A11820712
:100010003F34063406345B345B344F3466346D341D
:100020007C34013402340334043405340634073498
:10003000FF34FF34FF34FF34003400340034003424
:1000400000341330840000080319372801308D0074
:10005000BF308C0064008C0B2A288D0B28284A3076
:100060008C008C0B312800006400800B26280034A3
:10007000C830930021203F30900010088600860988
:10008000C8309300212006309000100886008609B1
:10009000C8309300212006309000100886008609A1
:1000A000C830930021205B3090001008860086093C
:1000B000C830930021205B3090001008860086092C
:1000C000C830930021204F30900010088600860928
:1000D000C830930021206630900010088600860901
:1000E000C830930021206D309000100886008609EA
:1000F000C830930021207C309000100886008609CB
:1001000002309200FA3093002120920B8228B1280D
:10011000323092001108FF3A7F39860012089203AC
:1001200000380319A32805080E398C000E300C0284
:1001300003199C28323092000130930021201108CD
:10014000860086098E28282984011F3083056500D2
:100150000030660086016430930021208E018F01FB
:1001600038280E0804208D009100110886008609A9
:1001700005080E398C000E300C02031928290E08D0
:100180008C000319E42801300C020319EA2802301C
:100190000C020319F82803300C020319F828043064
:1001A0000C020319F82805300C020319F828063050
:1001B0000C020319F82807300C020319F82808303C
:1001C0000C020319F8281A290519E82801308E00B5
:1001D0008F011A298518F1288F08031DF128023094
:1001E0008E008518F72801300F0203198E011A2995
:1001F00002300E02031D01298518012901308E00ED
:100200001729851D8E0A051D8E0303300E02031C5F
:100210000B29851C8E0102300E02031D17290519BA
:10022000172901300F02031D172901308E000130FC
:100230008F001A2909300E02031C202908308E0075
:100240000E0804208D009100110886008609882878
:04025000B828630067
:02400E000200AE
:084000000200090000000900A4
:0A42000001000000010000000100B1
:00000001FF
